:100000000C9495010C94CD010C94CD010C94CD0170
:100010000C94CD010C94CD010C94CD010C94CD0128
:100020000C94CD010C94CD010C943C1A0C940E1B35
:100030000C9439150C94CD010C94CD010C94CD0188
:100040000C94CD010C94CD010C94CD010C94CD01F8
:100050000C94CD010C94C1150C94CD010C94CD01E0
:100060000C94CD010C94CD010C94CD010C94CD01D8
:100070000C94CD010C94CD010C94CD010C94CD01C8
:100080000C94CD010C94CD010C94CD010C94CD01B8
:100090000C94CD010C94CD010C94CD010C94CD01A8
:1000A0000C94CD010C94CD010C94CD01E503E50336
:1000B000110411047904A405A405A40597043005CE
:1000C000410541057B1BA21B9A1CA21B9A1CEE1B1F
:1000D000111C9A1C681C771C29001E001F002000A0
:1000E00021002200230024002500260027002D00E7
:1000F0002E002A004A002B0014001A0008001500E8
:1001000017001C0018000C00120013002F00300014
:1001100031004B00390004001600070009000A00F6
:100120000B000D000E000F0033003400000028000B
:100130004E00E1001D001B00060019000500110023
:1001400010003600370038000000E50052004D0076
:10015000E000E300E2000000000000002C000000CE
:100160000000E6000151E400500051004F0035004E
:100170003A003B003C003D003E003F004000410093
:1001800042004300440045004C00010039000100DA
:100190000100AA00A900A800010001004900010017
:1001A0004600470048000100010001000100010075
:1001B0000100010001000100010001000100010037
:1001C0000100000001000100010001000100010028
:1001D0000100010001000100010001000100000018
:1001E0000100010001000100010001000000000009
:1001F00000000100000000000100010001000100FA
:10020000010001000C03470031005F00360035009B
:1002100000001803470045004E0020004F004E002C
:10022000450020004C004C0043000000040309047A
:1002300009023B00020100A0FA09040000010301C9
:100240000100092111010001224000070581030876
:10025000000109040100010300000009211101004F
:1002600001226D0007058203200001120100020037
:1002700000000820E701000100010200010501095A
:1002800080A101850319012AB700150126B7009541
:100290000175108100C0050C0901A1018504190137
:1002A0002AA002150126A002950175108100C00543
:1002B000010906A1018506050719E029E7150025B2
:1002C000019508750181020507190029EF15002520
:1002D0000195F0750181020508190129059505753B
:1002E000019102950175039101C005010906A10163
:1002F000050719E029E71500250195087501810218
:100300009501750881010507190029FF150026FFD1
:1003100000950675088100050819012905950575E0
:10032000019102950175039101C011241FBECFEF09
:10033000DAE0DEBFCDBF04B603FE18C08091B00284
:100340009091B102A091B202B091B3028730904B6C
:10035000A740B04B59F41092B0021092B102109223
:10036000B2021092B302E0E0F8E3099511E0A0E0D8
:10037000B1E0EAE4FAE302C005900D92A838B107B3
:10038000D9F722E0A8E8B1E001C01D92A03BB20776
:10039000E1F70E9499110C94231D0C94000081E058
:1003A000089581E008950C94D10108950C94D5012D
:1003B0001F93CF93DF9300D000D01F92CDB7DEB74D
:1003C00049835A836B8330918B0189819A813111E2
:1003D00014C0662359F0222349F00E94DD07182F2C
:1003E000682F89819A810E94860703C00E94B10705
:1003F000182F69817A81812F04C00E94DD076981ED
:100400007A810F900F900F900F900F90DF91CF9106
:100410001F910C94010FFC01262F408151816281B4
:10042000738184810C94D80181E00895CF93DF9388
:10043000EC0160E00E940B02BE01DF91CF910C94B1
:10044000D6010C944A100C94461008950E94300670
:100450000E9425022FEF84E39CE0215080409040D1
:10046000E1F700C000000C94E7150F931F93CF93A2
:10047000DF938C0161E00E940B02EC01B8010E9445
:10048000D3018823F1F1B801CE010E949213882391
:10049000C1F1B801CE010E94A611882391F1B801E3
:1004A000CE010E94EE12882361F1F8018281882337
:1004B00009F1CB358DE5D807C1F050F4C115FCE545
:1004C000DF0781F0CF3DDC45A9F40E94140D19C06F
:1004D000CC35EDE5DE0761F0CD35DD4559F40E9400
:1004E000570C08C00E9426020CC00E94600C02C07B
:1004F0000E94630CC801DF91CF911F910F910C9462
:10050000CF0180E0DF91CF911F910F9108950E945C
:100510001B150C94A0020E94A3020C9421150895AF
:100520000C948F0281E008950C9492020895CF9369
:10053000C82F0E9490028C2F0E949402CF910895A0
:1005400080E00C9497020E94EE130C9497020E9494
:10055000EE1390918A01891721F080938A010C94FF
:1005600097020895CF93DF93CDB7DEB72B970FB6E1
:10057000F894DEBF0FBECDBF4F83588769877A8757
:100580008B8761110E94A30B9E012F5F3F4F86E076
:10059000F90111928A95E9F785E0FE013796D901B4
:1005A00001900D928A95E1F789819A814C815D8154
:1005B000452B31F09F3F31F491E08F3F19F403C098
:1005C00091E001C090E090FF09C049815A816B81A0
:1005D0007C818D819E810E94C40A05C0C9010E9450
:1005E00014028111F2CF2B960FB6F894DEBF0FBE26
:1005F000CDBFDF91CF910895FC01808191810E9450
:100600001F080895CF93882309F448C0C82F8CEFA2
:100610008C0F813AD0F46C2F8091020190910301EC
:100620000E945614882349F06C2F8091020190910A
:1006300003010E94E1140E94C50B6C2F80910201FE
:10064000909103010E94D6140CC080E28C0F883078
:1006500058F4C77081E001C0880FCA95EAF70E947C
:10066000860BCF910C94C50BEBE5EC0FE33040F417
:10067000F0E0E15CFE4F808190E0CF910C94141487
:10068000C85AC73158F4EC2FF0E0EE0FFF1FEF5EB1
:10069000FE4F80819181CF910C942A14CF910895BF
:1006A000882349F1682F8CEF860F813A38F48091C6
:1006B0000201909103010E94E1140CC080E2860FB8
:1006C000883050F4677081E001C0880F6A95EAF7BE
:1006D0000E948C0B0C94C50B8BE5860F833020F4A5
:1006E00080E090E00C941414685A673120F480E0A4
:1006F00090E00C942A1408951F93CF93DF93182F42
:10070000EB010E940203209741F08FE99FE00197DF
:10071000F1F700C000002197F6CF812FDF91CF9134
:100720001F910C945003893319F060E070E002C00F
:1007300060E570E00C947C03882321F00E94860B16
:100740000C94C50B0895882321F00E948C0B0C9407
:10075000C50B0895CF92DF92EF92FF920F931F93F4
:10076000CF93DF937C01D62FC72FFC011281058127
:1007700002950F700E947C0B8823B9F01123A9F019
:100780008C2F807F803421F080E28D0F883068F0DC
:1007900080918A0282FD09C082E00E94250C0E949D
:1007A0007C0B91E0D82ED92601C0D12CCC2EC2943E
:1007B0008FE0C8228C2D90E08C30910508F0C4C1E8
:1007C000FC01EA5AFF4F0C94CE1C8C2F807FCF7017
:1007D000882311F0C295C07F112399F0CC2309F42E
:1007E0009FC180E28D0F883010F0D11104C08C2F92
:1007F0000E94860B03C08C2F0E94960B0E94C50B93
:100800008FC18D2F0E945003CC2309F49DC180E23B
:100810008D0F883038F1DD2329F18C2F0E949C0B3D
:1008200024C08C2F807FCF70803211F0C295C07FA2
:10083000DD2319F0D130A1F13DC080918A0282FF01
:1008400017C0112349F0CC2329F08C2F0E94860B6E
:100850000E94C50B80E065C180E00E945003CC235C
:1008600009F472C18C2F0E948C0B0E94C50B6CC1C5
:10087000112371F0002341F0013031F40E94A60BE6
:100880008C2B0E94AE0B60C10E94A60B8C2B1DC04E
:10089000002319F0013009F457C10E94BB0B25C099
:1008A000112321F0063008F04FC10EC0053008F0CA
:1008B0004BC11BC0112361F0002331F0F70185818A
:1008C00080FF2EC18F7085838C2F0E949C033CC1BA
:1008D000002359F0D93309F034C1FFEF07EE13E0DC
:1008E000F15000401040E1F72AC18C2F0E94A30371
:1008F0002BC18C2F86958695837019F0813061F01D
:1009000023C1112321F08D2F9C2F937002C080E012
:1009100090E00E94141420C1112321F08D2F9C2FF0
:10092000937002C080E090E00E942A1415C18C2FC1
:10093000837009F047C011110BC12D2F2295269508
:100940002770220F220F6D2F6F70862F90E0A0E08E
:10095000B0E0022E04C0880F991FAA1FBB1F0A9483
:10096000D2F7D4FF10C04FE050E060E070E004C068
:10097000440F551F661F771F2A95D2F74095509553
:100980006095709503C040E050E0BA01C695C695E9
:10099000C3708A019B01082B192B2A2B3B2BC90101
:1009A000B801C23049F058F4C13019F00E949C06D9
:1009B000CFC00E948A06CCC00E94AE06C9C00E9469
:1009C0008806C6C0112319F08C2F817001C086954E
:1009D000882309F4BDC02D2F229526952770220F5C
:1009E000220F6D2F6F70862F90E0A0E0B0E0022EF6
:1009F00004C0880F991FAA1FBB1F0A94D2F7D4FF07
:100A000010C04FE050E060E070E004C0440F551F9C
:100A1000661F771F2A95D2F740955095609570957F
:100A200003C040E050E0BA01C695C695C3708A0184
:100A30009B01082B192B2A2B3B2BC901B801C23073
:100A400049F058F4C13019F00E94610781C00E943A
:100A50004F077EC00E9473077BC00E94C20678C009
:100A6000CF70112339F08C2F0E94E8068D2F0E9441
:100A70009C036EC08D2F0E94A3038C2F0E94090738
:100A800067C0D23F21F128F4D03F41F0D13FC1F0FF
:100A900043C0D33F19F1D43F79F03EC0112341F058
:100AA000053008F051C08C2F8F710E942E074CC06A
:100AB000063008F049C0F7CF80918A0282FF18C043
:100AC000112339F08C2F8F710E94E8063DC011234D
:100AD000C9F38C2F8F710E94090736C0112329F0AA
:100AE0008C2F8F710E94D3062FC00E94CE062CC07F
:100AF000112349F0CF718C2F0E94E80663E08C2F00
:100B00000E940A0C21C081E00E94250C0230E0F016
:100B100082E00E94250C18C0112331F0002391F2CD
:100B20008D2F0E94020310C0002399F2D93349F49B
:100B30001FEF27EE33E0115020403040E1F700C0B6
:100B400000008D2F0E94500388EF8C0D843020F41C
:100B50000E94EE130E949702DD20C9F00E94780BDC
:100B600080FD15C0F70112820E94720B0E94E806F8
:100B7000C7010E94E8050E94720BDF91CF911F917F
:100B80000F91FF90EF90DF90CF900C940907DF91C9
:100B9000CF911F910F91FF90EF90DF90CF9008952C
:100BA0000F931F93CF93DF93EC01688179818A8142
:100BB0000E942A088C010E9485070E947606B801CF
:100BC000CE010E94AA03DF91CF911F910F9108954A
:100BD000CF93DF93EC01988189812B813C81232B7A
:100BE00031F08F3F31F481E09F3F19F403C081E081
:100BF00001C080E080FD1DC0CE010E943502811140
:100C000010C00E947C0B8823A1F08A81882389F080
:100C100080918A0282FD0DC082E0DF91CF910C9419
:100C2000250CCE010E94D005CE01DF91CF910C940E
:100C30001602DF91CF91089580E090E00E94141495
:100C400080E090E00E942A140E94A30B0C94C50B34
:100C500080910201909103010E94EC140C941C06F7
:100C60000E94930B0C94280692959F70963079F011
:100C700010F4925001C09A50923068F4803F69F0AD
:100C800018F4883E40F409C0843F29F406C0883E29
:100C900020F0813F11F080E0089581E00895FC018B
:100CA000808191810E941F080E9434060895CF938D
:100CB000DF9300D000D01F92CDB7DEB70F900F901A
:100CC0000F900F900F90DF91CF910895CF93DF9306
:100CD00000D000D000D0CDB7DEB726960FB6F8947E
:100CE000DEBF0FBECDBFDF91CF9108950895089567
:100CF0000C9477060C9478060E947A066093C201E1
:100D00007093C3018093C4019093C5010C941C0699
:100D10000C947C060F931F930091C2011091C301A4
:100D20002091C4013091C501602B712B822B932B34
:100D30001F910F910C947C060F931F930091C20199
:100D40001091C3012091C4013091C501602371232A
:100D5000822393231F910F910C947C060F931F9372
:100D60000091C2011091C3012091C4013091C501CD
:100D700060277127822793271F910F910C947C067F
:100D80000C9477060E94C0066093BE017093BF0169
:100D90008093C0019093C1010C941C0660E070E048
:100DA000CB010C94C2060F931F9341E050E060E02A
:100DB00070E08A019B0104C0000F111F221F331F26
:100DC0008A95D2F7C901B8011F910F910C94C20600
:100DD0000F931F9341E050E060E070E004C0440FC7
:100DE000551F661F771F8A95D2F78091BE0190919B
:100DF000BF01A091C001B091C1018A019B01082BE4
:100E0000192B2A2B3B2BC901B8011F910F910C9470
:100E1000C2060F931F9341E050E060E070E004C011
:100E2000440F551F661F771F8A95D2F7409550953E
:100E3000609570958091BE019091BF01A091C00115
:100E4000B091C1018A019B01082319232A233B2366
:100E5000C901B8011F910F910C94C2060F931F9303
:100E600041E050E060E070E004C0440F551F661F91
:100E7000771F8A95D2F78091BE019091BF01A09112
:100E8000C001B091C1018A019B01082719272A27B7
:100E90003B27C901B8011F910F910C94C2060F9313
:100EA0001F930091BE011091BF012091C0013091AC
:100EB000C101602B712B822B932B1F910F910C94EE
:100EC000C2060F931F930091BE011091BF012091A4
:100ED000C0013091C10160237123822393231F91AC
:100EE0000F910C94C2060F931F930091BE011091B5
:100EF000BF012091C0013091C10160277127822775
:100F000093271F910F910C94C20608952FE0929F92
:100F1000800D1124E82FE695E695E695877051E05F
:100F200001C0550F8A95EAF785E0E89FF00111248A
:100F3000E457FE4F20E030E070E04081CB01022E0C
:100F400002C0969587950A94E2F78170819584276F
:100F50008523842781932F5F3F4F2530310569F723
:100F600008952FE0929F800D1124682F6695669555
:100F70006695982F977085E0689FB001112440E036
:100F800050E080E0FB01E40FF51FE457FE4F2081A5
:100F900030E0092E02C0369527950A94E2F72170B9
:100FA0003327042E01C0220F0A94EAF7822B4F5FE9
:100FB0005F4F4530510531F70895BF92CF92DF92D0
:100FC000EF92FF920F931F93CF93DF938C01C0900A
:100FD000BE01D090BF01E090C001F090C1018091AE
:100FE000C2019091C301A091C401B091C501C82A6A
:100FF000D92AEA2AFB2ACFE1D0E0D701C6010C2E7C
:1010000004C0B695A795979587950A94D2F780FD69
:1010100004C0219790F7B12C07C0BC2EB8018C2FCB
:101020000E94140F0197A9F38B2DDF91CF911F918F
:101030000F91FF90EF90DF90CF90BF900895CF93E6
:10104000DF93EC010E94DD07BE010E94140FDF91C7
:10105000CF9108951F93CF93DF93EB0190918B0174
:10106000992321F0CB010E941F0813C0882349F067
:10107000CB010E94DD07182F682FCE010E94860742
:1010800004C0CB010E94B107182FBE01812F0E941E
:10109000140FDF91CF911F9108951F93CF93DF938A
:1010A000C091C60116E08091C701C81799F0D0E041
:1010B0001C9FF0011D9FF00D1124E853FE4F40814D
:1010C000518162817381848195810E946606219697
:1010D000C770E9CFDF91CF911F9108954091F8013A
:1010E0005091F9016091FA017091FB018091FC012E
:1010F0009091FD010C946606EF92FF920F931F935F
:10110000CF93DF938091FD0182958F7009F065C0C8
:101110008091FA01882309F460C08091C601F090A3
:10112000C7011091F8010091F9016091FB017091E4
:10113000FC0191E01F3F09F090E0C0910001D091C7
:101140000101292F96E0E92E8F1509F446C061159B
:10115000710521F00F3F21F030E003C031E001C004
:10116000322F90E030FD36C0E89EF001E99EF00D90
:101170001124DF01A853BE4F11963C9111973013F3
:1011800029C03C91311326C012963C91129731111F
:1011900021C013964D915C911497461B570B4C1729
:1011A0005D07C0F48091FD018F7080618093FD0127
:1011B000E353FE4F80818F708061808388EF91E0E0
:1011C0000E94E805DF91CF911F910F91FF90EF9062
:1011D0000C944D0801968770B7CFDF91CF911F9186
:1011E0000F91FF90EF9008959F92AF92BF92CF9290
:1011F000DF92EF92FF920F931F93CF93DF93CDB7C0
:10120000DEB761970FB6F894DEBF0FBECDBF8C017D
:1012100085E0F801DE011D9601900D928A95E1F7B7
:10122000D8011296EC909091F801E091F90120918B
:10123000FB013091FC012115310531F0EF3F31F414
:1012400081E09F3F19F403C081E001C080E0B82F26
:10125000B1709B2E80FD47C1D8014C9111965C91D5
:1012600011971396AD90BC90149788EFC82E81E02B
:10127000D82EF090FA01B501621B730B209100018A
:1012800030910101FF2009F4D9C08091FD0162175E
:10129000730708F095C0282F207F09F052C05E1315
:1012A00013C0491311C0FE2CE1100EC08F70806175
:1012B0008093FD010E946E08C6010E94E80580919E
:1012C000FD01F80185834DC1AB2831F05F3F31F45A
:1012D00081E04F3F19F403C081E001C080E080FD50
:1012E00003C081E08E2502C080E090E0F82FF1700D
:1012F000FF2E80FF1CC08091C6012091C70136E0FF
:10130000821709F40BC190E0389FF001399FF00D6E
:101310001124E853FE4F6181561306C060814613C5
:1013200003C06281E61203C001968770E9CFFE2CEC
:10133000EE2009F416C18091FD0181608093FD01CA
:1013400054C05E1306C0491304C0E11002C0F80186
:1013500099C0C8010E944F06882361F1EE2051F127
:101360002091FD01822F82958F7090E0029774F09A
:101370008091F8019091F90198878F831986BB8637
:10138000AA862C87CE0107960E94E80586E0F80120
:10139000A8EFB1E001900D928A95E1F70E947C08D8
:1013A0000E946E080AC05E1711F1C8010E944F0624
:1013B00081112CC0C8010E94E805FF24F394D1C01C
:1013C000282F207F81F77A2DB98AA88A6E2D8989E6
:1013D0000E94570688EF91E00E94E80586E0D6015A
:1013E0001D928A95E9F70E946E08F12CBAC0491344
:1013F000DCCFE110DACFF8018583C8010E94E8054F
:1014000086E0D6011D928A95E9F7ABC0EE2091F2F5
:101410002091FD01822F82958F7090E002970CF44D
:10142000B5CF8091F8019091F9019A8389831B824D
:10143000BD82AC822E83CE010196A6CF62177307C0
:1014400008F044C0FE2CEE2009F4B4CF5E1330C087
:1014500049132EC02091FD0120FD21C0822F8295CD
:101460008F70482F50E041155105C9F0F8012583D0
:101470004F30510541F08F5F982F9295907F822FCA
:101480008F70892B8583C8010E94E80586E0F801EA
:10149000A8EFB1E001900D928A95E1F73CC086E09B
:1014A000F801A8EFB1E001900D928A95E1F759C0DB
:1014B000C8010E944F06811169CF8091FD018160B2
:1014C0008093FD01C8010E94E8054BC07A2DB98ABE
:1014D000A88A6E2D89890E94570686E0D6011D9242
:1014E0008A95E9F718C0EE2009F464CFC8010E947C
:1014F0004F06F82E882309F45DCF86E0F801A8EFA7
:10150000B1E001900D928A95E1F788EF91E00E9499
:10151000FC020E947C080E946E0823C04D875E87F3
:101520008D859E850E941F08292F22952F702230BD
:1015300028F49F7039F0811105C00BC0243028F4C5
:101540009F7049F4805E883020F0C8010E94E80551
:101550009F2CF92C06C0D80115969C91907F91F78D
:10156000F8CF8F2D61960FB6F894DEBF0FBECDBFBA
:10157000DF91CF911F910F91FF90EF90DF90CF906F
:10158000BF90AF909F9008951F93CF93DF93CDB7F7
:10159000DEB72C970FB6F894DEBF0FBECDBF4F83DA
:1015A000588769877A878B879C87CE0107960E9428
:1015B000F4088823D1F09F8188852A853B85232BD9
:1015C00031F08F3F31F481E09F3F19F403C081E097
:1015D00001C080E080FD47C04F81588569857A85CC
:1015E0008B859C850E9466063EC086E0FE0137968C
:1015F000DE01119601900D928A95E1F7FF81E88551
:101600006A857B856115710531F0EF3F31F481E02A
:10161000FF3F19F403C081E001C080E080FD23C0DA
:101620002091C70130E0C901019687709927409148
:10163000C60150E084179507F1F1F983EA837D83B1
:101640006C8396E0929FD001939FB00D1124A85314
:10165000BE4FFE01319601900D929A95E1F780936D
:10166000C7010E944D0816E08091C6019091C70104
:10167000891771F1189FC001112488539E4F0E9451
:10168000F408882329F1E091C6011E9FF00111247E
:10169000E853FE4F4081518162817381848195813D
:1016A0000E9466068091C60190E001968770992796
:1016B0008093C601D9CF0E9430061092C7011092C4
:1016C000C601E8EFF1E086E0DF011D928A95E9F7B7
:1016D0002C960FB6F894DEBF0FBECDBFDF91CF9131
:1016E0001F91089580911E02859585958595089591
:1016F00080911E028770089590911E02977081E07C
:1017000009F480E00895809141020895909141028A
:10171000892B8093410208958095909141028923FD
:1017200080934102089510924102089590914002E1
:10173000892B8093400208958095909140028923DF
:1017400080934002089510924002089580911F02F4
:10175000089508950C94A90B0C94AA0B90918A02F9
:1017600092FD08C090911F02981721F080931F02EC
:101770000C94AC0B089580911F02882329F01092DD
:101780001F0280E00C94AC0B0895CF93DF93E0919F
:101790000201F0910301809141028083E0910201F6
:1017A000F0910301908180914002892B8083809188
:1017B0001F02882381F0E0910201F09103019081E2
:1017C000892B808380910201909103010E94401433
:1017D00081110E94BB0BC0910201D091030140E234
:1017E00050E06EEF71E0CE010E94D41C892B69F0AD
:1017F00080E2FE01AEEFB1E001900D928A95E1F733
:10180000CE01DF91CF910C94FA13DF91CF9108951F
:101810000C94A90B90918A0292FD10C098E0899FC8
:1018200090011124262B20931E020E94E80680912D
:101830001E028595859585950C94080C0C94E806F8
:1018400010921E0280E00C94080C20911E028095DC
:10185000822380931E02982F977099F430E0482FCE
:10186000082E000C550B2417350759F090918A0269
:1018700092FD07C08595859585950E9409070C9472
:10188000200C089590918A0292FB222720F92817B4
:1018900069F080FB92F990938A028091890290917D
:1018A0008A020E94900C82E00C94250C089580918D
:1018B0008A0282FB882780F991E089270C94420CE8
:1018C00081E00C94420C80E00C94420C6FEF7FEFAF
:1018D00080E090E00C940D1D80E090E00E94E91CF7
:1018E00021E0893E9E4F09F020E0822F089582E09A
:1018F00090E00C94E11C83E090E00C94E11CCF9309
:1019000084E090E00E94E11CC82F82E290E00E94F7
:10191000E11C2C2F30E0A901582BCA01CF9108956A
:10192000CF93C92F682F84E090E00E94EF1C6C2FAA
:1019300082E290E0CF910C94EF1CAB01BC018FE0F0
:1019400090E00C94011DAB01BC0183E190E00C948C
:10195000011D60E070E0CB010C94A30C60E070E02E
:10196000CB010E949D0C0C94A90C69EE7EEF80E0E7
:1019700090E00E940D1D60E082E090E00E94EF1C6C
:1019800060E083E090E00E94EF1C1092C201109290
:10199000C3011092C4011092C50160E084E090E0A0
:1019A0000E94EF1C60E082E290E00E94EF1C60E089
:1019B00085E090E00E94EF1C60E086E090E00E94ED
:1019C000EF1C6FEF87E090E00E94EF1C40E050E0DA
:1019D000BA0188E090E00E94011D60E08DE090E097
:1019E0000E94EF1C40E050E0BA0188E190E00E94C4
:1019F000011D60E087E190E00E94EF1C40E050E0B4
:101A0000BA018CE190E00E94011D60E070E080E28C
:101A100090E00E940D1D40E050E0BA0188E190E0A6
:101A20000E94011D0C94AE0C0C94B50C682F8EE036
:101A300090E00C94EF1C0E94A615609350027093E6
:101A40005102809352029093530260934C02709320
:101A50004D0280934E0290934F02089585B780689F
:101A600085BF85B7806885BF089581E008950C948F
:101A7000350D08950C94390D0C94390D0C943C0DD2
:101A80000C94390D0C94400D0C94390D0E942E0DC0
:101A900080EF9FE00E94E4130E94440D0C94420DDD
:101AA0000E943A0D0C94390D0E940D100C94960270
:101AB0000E9491150E94F2100E94540D0C943E0D4C
:101AC0005F926F927F928F929F92AF92BF92CF92CE
:101AD000DF92EF92FF920F931F93CF93DF93CDB7D7
:101AE000DEB72A970FB6F894DEBF0FBECDBF0E94B7
:101AF0000711C82E81110E941B0D32E4832E32E0A3
:101B0000932E00E010E0502E802F0E9431105C01D7
:101B1000F401619071904F01682679266114710477
:101B2000B1F40F5F1F4F0530110569F78FEF8983FF
:101B30008A831B820E949A158160782F9D838C83F3
:101B400049815A816B818D810E94B2023AC0809195
:101B5000540281FD0E943A10D12CEE24E394F12C22
:101B6000C3018E219F21892B29F10E94370D8823E3
:101B7000A9F0DE825F82AE20BF2081E0AB2809F4AD
:101B800080E088870E949A158160782F9A878987DC
:101B90004E815F8168858A850E94B202000F111F05
:101BA000F801EE5BFD4F80819181E826F926F182F4
:101BB000E08207C0D394EE0CFF1CFFE0DF12D0CF11
:101BC000B0CF81E0C11001C080E02A960FB6F89432
:101BD000DEBF0FBECDBFDF91CF911F910F91FF9060
:101BE000EF90DF90CF90BF90AF909F908F907F90BD
:101BF0006F905F9008950E94600D0C94A702CF93A0
:101C0000DF930E94190FEC01811522E59207E8F598
:101C1000811531E5930708F0B6C0883E910528F597
:101C2000803E910508F0E9C0883A910570F4853A44
:101C3000910508F07AC08130910509F473C008F469
:101C4000D9C0049708F0D9C0D5C08F3B910508F0E2
:101C5000D1C0C85AD0E0CC0FDD1FCE5BDE4F09905B
:101C6000D881C02DCE019464C9C0811540E5940788
:101C700008F069C0811550E4950708F060C09A9596
:101C800081159F4108F4B9C0B5C0811536E59307A9
:101C900028F5811545E5940708F092C0811554E5B3
:101CA000950708F087C0AC0143705527282F26956B
:101CB0002695C115D34508F06CC081E090E002C0C4
:101CC000880F991F4A95E2F740E2249F9001112462
:101CD000EC01C22BD32BCE019C6890C081152AE564
:101CE000920780F4811539E5930708F072C08115D9
:101CF00048E5940708F47EC0D82FCC27CE01806F2A
:101D0000906A7CC090568115904208F073C08D2F68
:101D10008F710E94AD0FDD27D0628F71AE01582BFD
:101D2000CA016CC081E090E069C0C55AD0E0C059DA
:101D3000DE4F8881C82FD0E0CE0190645FC0DF7095
:101D4000CE01906A5BC074E0969587957A95E1F72D
:101D5000282F23703C2F337081E090E002C0880F61
:101D6000991F3A95E2F79C68AC01522B9A019C2F7F
:101D70009F709695969550E2959FE0011124C901B8
:101D80008C2B9D2B3BC0D82FCC27CE01816F906A26
:101D900035C081E090E002C0880F991F4A95E2F7B4
:101DA00050E2259F90011124EC01C22BD32BCE01D0
:101DB0009A6824C0D82FCC27CE01846F906A1EC0A9
:101DC0000E94AD0F8F7190E0D82FCC27CE0190628A
:101DD00015C08F700E94AD0F94E0D695C7959A9567
:101DE000E1F7CF70D0E0DC2FCC27D0699E01282B03
:101DF000C90104C080E090E001C0CE01DF91CF9125
:101E000008952BE4829FC0011124FC012FE0729FF2
:101E1000E00DF11D1124E60FF11DEE0FFF1FE8523A
:101E2000FF4F8591949108950E94010F0E94FF0D2C
:101E300008958238910569F1B0F48133910509F470
:101E40006DC048F48932910509F463C08A32910566
:101E500009F469C008958533910509F455C08933A3
:101E60009105B9F00895833E910569F138F4803EFB
:101E70009105B1F0823E910509F10895863E9105E4
:101E8000A9F1873E9105B9F1843E910509F064C03E
:101E900023C02091890220FD4FC021FD4DC008952F
:101EA0008091890280FD44C080918A0280FF44C0F5
:101EB0008091890284FD42C083EE4DC080918902E9
:101EC00082FF38C0F5CF8091890282FD33C08091B6
:101ED0008A0280FD31C0ECCF80918A0281FF32C03E
:101EE0008091890284FD2AC087EE35C080918902E5
:101EF00083FF26C0F5CF8091890283FD21C08091A8
:101F00008A0281FD1FC0ECCF8091890285FD1CC033
:101F10001DC08091890285FD19C016C0809189027B
:101F200086FD16C017C08091890286FD13C010C0BF
:101F300089E311C082EE0FC080EE0DC080E00BC0BF
:101F400086EE09C084EE07C089E205C085E303C0C0
:101F50008AE201C081E390E008959091890292FFA6
:101F60000DC0282F2871283019F4877F846006C09F
:101F7000282F2471243011F48B7F886093FF0DC0CB
:101F8000282F2871283119F4877E846106C0282FF4
:101F90002471243111F48B7E886120918A0220FF04
:101FA0000DC0382F3871383019F4877F816006C032
:101FB000382F3171313011F48E7F886021FF0DC0D0
:101FC000282F2871283119F4877E816106C0282FB7
:101FD0002171213111F48E7E886194FD877E0895F0
:101FE00080E008950C94660C0E9407112FEF86E79D
:101FF00091E0215080409040E1F700C000000E9435
:10200000071180E00E94311080FF04C00E94F20F8F
:102010000C94E71508950C94F40F0E946C0C811138
:1020200002C00E94140D0E94770C809354020E94FB
:102030007F0C90938A02809389020E940B100E9469
:102040007B0C682F70E080E090E00E948806609131
:10205000BE017091BF018091C0019091C1010C94AB
:10206000C006E82FF0E0EE0FFF1FEB56FD4F80811A
:1020700091810895089580EA8A95F1F7089500C046
:1020800008950C943B1008950C9443100C94441044
:102090000C9443100C944810F894E82FE295EF70DC
:1020A000F0E031A1282F2F7081E090E001C0880F6F
:1020B0002A95EAF7982F9095932391A392A1892BC3
:1020C00082A3789408950F931F93CF93DF93C2E870
:1020D000D1E089918F3F11F00E944C1081E0C73808
:1020E000D807B9F7C3E7D1E002E811E089918F3F43
:1020F00011F00E944C100C171D07C1F7DF91CF9112
:102100001F910F910895BF92CF92DF92EF92FF92AD
:102110000F931F93CF93DF938C01C62FD0E0CE0196
:102120008E579E4F6C01FC0190819F3F09F450C077
:10213000B62EF894E92FE295EF70F0E081A19F7040
:1021400021E030E001C0220F9A95EAF7822B81A3AB
:1021500082A12095282322A378940E943F10E3E7D0
:10216000F1E042E851E021E030E0E12CF12C619116
:102170006F3F89F0A62FA295AF70B0E090968C913A
:1021800090E06F7002C0959587956A95E2F780FDA3
:1021900002C0C90102C080E090E0E82AF92A220FBB
:1021A000331F4E175F0719F7F60180818F3F11F03B
:1021B0000E944C1061E0E114F10409F460E08B2D01
:1021C0000E944110CC0FDD1FC00FD11FF982E882A1
:1021D000DF91CF911F910F91FF90EF90DF90CF9003
:1021E000BF9008950E9463108AE0E5E9F2E0DF0104
:1021F000982F1D929A95E9F7EBE8F2E0DF011D9226
:102200008A95E9F785E00E9452110C942102FF9211
:102210000F931F93CF93DF93CDB7DEB72A970FB6F7
:10222000F894DEBF0FBECDBF8E010F5F1F4F8AE057
:10223000F80111928A95E9F7F12C6F2DC8010E94DF
:102240008310F394F5E0FF12F8CF4AE050E0B801B4
:102250008BE892E00E94D41CFF24F394009709F4C9
:10226000F12C892B41F08AE0F801ABE8B2E0019053
:102270000D928A95E1F72F2D45E065E972E08BE834
:1022800092E00E9453110E9423028F2D2A960FB6CE
:10229000F894DEBF0FBECDBFDF91CF911F910F919C
:1022A000FF9008950895FF920F931F93CF93DF93AC
:1022B000F82E092F162FD72FC42F222349F081E0A3
:1022C000809357020E949A1590935602809355026C
:1022D000809157028823D9F080915502909156023F
:1022E0000E94B215059798F0EF2DF02FA12FBD2F6A
:1022F00080E090E04C2F50E08417950734F4219152
:1023000031912D933D930196F7CF10925702DF91B3
:10231000CF911F910F91FF9008950E9494170E94F2
:10232000580D0C94A0170E94A4170E94FB0D0C944A
:10233000BE170E9438150E947B170E94460D0E940E
:102340008D110E9493110E94500DFBCFCF93DF930C
:10235000EC01FB018281882309F43CC1C430FDE516
:10236000DF0760F4CB3F9CE5D90788F49E0122503B
:102370003C452431310508F02EC109C0C236EDE5D7
:10238000DE0729F0C63AFDE5DF0709F024C10E9407
:102390007F0C90938A0280938902C1318CE5D80723
:1023A00009F4C6C008F042C0C930ECE5DE0709F404
:1023B0009BC000F5C5308CE5D80709F485C078F4DA
:1023C000C330ECE5DE0709F478C008F07AC0C2300B
:1023D000DC4509F0F5C0809189028160EFC0C7300B
:1023E0009CE5D90709F478C008F07AC08091890289
:1023F0008061E4C0CD30FCE5DF0709F487C058F404
:10240000CB309CE5D90709F479C008F07BC08091F6
:10241000890288606FC0CF30FCE5DF0709F480C017
:1024200008F082C080918902877FC8C0CE3F9CE5BA
:10243000D90709F471C000F5C531FCE5DF0709F4DF
:1024400085C068F4C3319CE5D90709F475C008F06C
:1024500095C00E943006809189028F77AFC0CC3F33
:10246000FCE5DF07A9F108F054C0CB3FDC4509F0DB
:10247000A7C080918A0240C0C230EDE5DE0709F4B2
:1024800089C058F4C1158DE5D80709F45AC008F081
:1024900069C080918A0282602FC0C236EDE5DE07F6
:1024A00009F47CC0C63AFDE5DF0709F481C0C330FA
:1024B000DD4509F085C080E06EC0809189028260B0
:1024C0007DC08091890216C080918902886076C0A3
:1024D00080918A0282604FC08091890280626EC0C2
:1024E0008091890280646AC00E94300680918902CE
:1024F000806864C0846062C081603DC08091890250
:102500008E7F5CC0809189028D7F58C08091890246
:1025100016C080918A0218C080918A028D7F2BC0DC
:10252000809189028F7E4AC0809189028F7D46C04A
:10253000809189028F7B42C080918902877F8B7F47
:102540003DC080918A028D7F8E7F15C08091890267
:1025500082FB222720F991E0922790FB82F990FBE1
:1025600083F92CC080918A02982F909591708E7F6C
:10257000892B90FB81F980938A0222C00E94300649
:102580008091890287FB222720F991E0922790FB16
:1025900087F914C081E00E94160D12C08091890253
:1025A00084FB222720F991E0922790FB84F906C052
:1025B00080918902982F909590FB80F980938902F1
:1025C0008091890290918A020E94900C0E943006AC
:1025D00080E001C081E0DF91CF910895CF93DF9338
:1025E00086319C4541F5EB010E94830B982F8A812F
:1025F0002091020130910301882379F09A7A81E0D9
:1026000009F480E080935802911102C069E201C090
:1026100065E3C9010E94D6140AC080915802811155
:1026200002C069E201C065E3C9010E94E1140E9491
:10263000C50B80E001C081E0DF91CF9108950F9339
:102640001F93CF93DF93C42FD22FFC018281882365
:10265000C9F040935B020E949A1590935A028093AE
:10266000590280E28C0F883008F057C0C77081E0B3
:1026700001C0880FCA95EAF7DF91CF911F910F91A2
:102680000C949C0380915B02481330C080915902E6
:1026900090915A020E94B215883C910538F510E2DB
:1026A0001D0FCD17B9F080E28C0F883040F4C77051
:1026B00081E001C0880FCA95EAF70E94A303183091
:1026C00028F581E09D2F977001C0880F9A95EAF751
:1026D0000E949C03802F0E9493031830F0F4D7705F
:1026E00081E001C0880FDA95EAF70AC080E28C0F1A
:1026F000883098F4C77081E001C0880FCA95EAF766
:10270000DF91CF911F910F910C94A303802FDF9144
:10271000CF911F910F910C949303DF91CF911F9153
:102720000F9108950F939C01CB01243F4CE5340792
:1027300031F188F4293DFCE53F07D9F02A3D4CE50D
:10274000340779F1283D3C45A9F506E221EE41EE3A
:1027500068ED7CE52BC0263FFCE53F07E1F0A8F0E3
:10276000273F3C4539F507E225EE46EE67EF7CE56D
:102770001DC007E225EE45EE69ED7CE517C006E2D7
:1027800021EE40EE64EF7CE511C007E225EE44EE59
:1027900065EF7CE50BC006E221EE42EE66EF7CE5DC
:1027A00005C008E221E045EE6AED7CE50E941F13BA
:1027B00080E008C0FC018281882319F010925B023E
:1027C00001C081E00F910895909389018093880161
:1027D000089590936102809360020895E0916002F1
:1027E000F0916102309721F00190F081E02D099481
:1027F00080E00895E0916002F0916102309799F0D5
:1028000020911001222359F02091890227FF07C04F
:10281000DC012C9111962C93119726E02C930280C9
:10282000F381E02D0994089520915E0230915F02BA
:102830002817390771F090935F0280935E02E09150
:102840006002F0916102309721F00680F781E02D5F
:102850000994089520915C0230915D022817390790
:1028600071F090935D0280935C02E0916002F091C0
:102870006102309721F00084F185E02D09940895DC
:10288000FC01329680911001882331F080918902F9
:1028900087FF02C09EE101C096E080E0915028F0E1
:1028A00021912223D9F38F5FF9CF0895662351F147
:1028B000209110012223E9F02091890227FF19C0FD
:1028C000462F4695469546954E31E0F4677021E0D7
:1028D00030E002C0220F331F6A95E2F7FC01E40FDB
:1028E000F11D828190E02823392381E0232B69F4B4
:1028F00009C0FC01329608962191621729F0E81769
:10290000F907D1F780E0089581E008959C01FC016A
:1029100032969FEF80E04191461789F09F3F19F46E
:10292000411101C0982F8F5F8630A9F79F3F39F082
:10293000F901E90FF11D97FDFA9562830895089555
:102940009C012A5F3F4FFC014281461301C0128265
:10295000019682179307B9F70895262F2695269595
:1029600026952E3168F4FC01E20FF11D677021E01D
:1029700030E001C0220F6A95EAF78281282B22837A
:102980000895262F2695269526952E3170F4FC0164
:10299000E20FF11D677021E030E001C0220F6A955F
:1029A000EAF720958281282322830895209110013F
:1029B000222329F02091890227FD0C94AD140C9458
:1029C000861420911001222329F02091890227FDED
:1029D0000C94C1140C94A01420911001FC013296A7
:1029E000222331F08091890287FF02C08EE101C06D
:1029F00086E0DF011D928A95E9F7089508950C9409
:102A0000FE1483E0809362020C94FF14811102C0D3
:102A100081E001C082E0809362020C94FF140C9468
:102A2000061581E0809362020C94FF140C9411153A
:102A300008950C9418150C9419150C9418150C94F1
:102A400018150C941815CF930E941F150E9407119A
:102A50000E941D15C0E08C2F0E943110892B29F493
:102A6000CF5FC530C1F780E001C081E0CF9108950C
:102A700008951F920F920FB60F9211248F939F9378
:102A8000AF93BF9380916302811113C080919F0225
:102A90009091A002A091A102B091A2024196A11D25
:102AA000B11D80939F029093A002A093A102B093C6
:102AB000A202BF91AF919F918F910F900FBE0F9087
:102AC0001F9018958091A702843031F10E948702EF
:102AD0001092630220E488E190E00FB6F894A89584
:102AE000809360000FBE2093600083B7817F846075
:102AF00083BF83B7816083BF7894889583B78E7FC7
:102B000083BF0FB6F894A895809160008861809388
:102B10006000109260000FBE08950E9430060C9471
:102B20008B0282E084BD93E095BD9AEF97BD8093C0
:102B30006E0008952FB7F89480919F029091A002A3
:102B4000A091A102B091A2022FBF08952FB7F894CF
:102B500060919F027091A0028091A1029091A202C7
:102B60002FBF08959C014FB7F89480919F029091D8
:102B7000A002A091A102B091A2024FBF821B930BB1
:102B8000089578941F920F920FB60F9211248F938D
:102B90009F93AF93BF9380919F029091A002A091C9
:102BA000A102B091A2020196A11DB11D80939F02C6
:102BB0009093A002A093A102B093A202BF91AF9103
:102BC0009F918F910F900FBE0F901F90189581E0ED
:102BD0008093E00080E28093D8001092C9008FE1DA
:102BE0009EE40197F1F700C0000087E090EBDC0164
:102BF0008093B0029093B102A093B202B093B3025B
:102C00009CE088E10FB6F894A895809360000FBE11
:102C100090936000FFCF8091870208950895CF932D
:102C2000DF9320911001222339F02091890227FFA0
:102C300003C060E222E002C068E021E02093E900E6
:102C40002FEF3091E800215035FD06C035ED3A9563
:102C5000F1F700002111F5CF2091E80025FF1DC0FC
:102C6000EC0180911001811105C040E050E068E066
:102C700070E003C070E040E050E0CE010E943018E8
:102C80008091E8008E778093E80080E2FE01A7E65D
:102C9000B2E001900D928A95E1F7DF91CF9108950E
:102CA0008093640270936602609365028091A7022C
:102CB000843001F582E08093E9008FEF9091E80085
:102CC000815095FD06C095ED9A95F1F700008111B0
:102CD000F5CF8091E80085FF0DC040E050E063E053
:102CE00070E084E692E00E9430188091E8008E77D0
:102CF0008093E8000895BC0184E00C945016BC0158
:102D000083E00C94501608958091A602811109C0A9
:102D10000E94C1190E941E1A8091E2008460809373
:102D2000E20008951092A60208950C941615609181
:102D3000A30281E0611101C080E00C940115909123
:102D4000A70281E0943009F080E06091A3020C9426
:102D5000061542E061EC81E00E943A1942E261EC22
:102D600082E00E943A199091A70281E0943009F024
:102D700080E06091A3020C940F158091A90283302A
:102D800009F461C030F4813071F0823009F49AC0E6
:102D900008958A3009F486C08B3009F46CC08930FC
:102DA00009F0A8C020C08091A802813A09F0A2C011
:102DB0008091E800877F8093E8008091AC02909139
:102DC000AD02892B21F460E287E692E003C060E067
:102DD00080E090E070E00E947B188091E8008B77A3
:102DE0008093E80008958091A802813209F082C0A2
:102DF0008091AC029091AD02029708F07BC0809167
:102E0000E800877F8093E8008091E80082FD05C09C
:102E10008091A7028111F8CF6DC02091F3008091BD
:102E2000F20090E0922B029731F48091F100813012
:102E300011F0863021F48091F10080938702809117
:102E4000E8008B7753C08091A802813A09F052C004
:102E50008091AC029091AD02892B09F04BC080911A
:102E6000E800877F8093E8008091E80080FFFCCF36
:102E70008091100136C08091A8028132D9F58091ED
:102E8000AC029091AD02892BA9F58091E800877F73
:102E90008093E8000E946F198091AA02809310012C
:102EA0000C9430068091A802813221F58091E800CF
:102EB000877F8093E8000E946F198091AB02809316
:102EC000880208958091A802813AA1F48091E800D7
:102ED000877F8093E8008091E80080FFFCCF80919D
:102EE00088028093F1008091E8008E778093E8005B
:102EF0000C946F19089584B7877F84BF0FB6F89438
:102F0000A8958091600088618093600010926000B5
:102F10000FBE90E080E80FB6F89480936100909324
:102F200061000FBE0C9411150E94C1190E941E1A57
:102F3000E2EEF0E080818460808378940C94B31C8E
:102F400084E091E00C94E9138091A7028530A9F404
:102F50008091A702853079F40E9462158091A502C4
:102F60008823B1F30E942315882391F30E941A1835
:102F70000E943006EDCF0C948D15089508950C94A1
:102F8000C117292F332723303105C9F060F42130D0
:102F9000310581F02230310509F044C08BE390E027
:102FA00020E332E043C021323105E1F02232310525
:102FB00049F138C082E190E02BE632E037C0992732
:102FC0008130910549F028F0029761F5E4E0F2E0E4
:102FD00005C0ECE2F2E002C0E2E1F2E0849190E0B0
:102FE0009F0124C06115710541F061307105D1F474
:102FF00089E090E02BE532E019C089E090E022E41E
:1030000032E014C06115710541F06130710551F471
:103010008DE690E02DE732E009C080E490E02AEEF2
:1030200032E004C080E090E020E030E0FA0131833B
:103030002083089580E189BD82E189BD09B400FE45
:10304000FDCF8091D8008F7D8093D8008091E000E3
:1030500082608093E0008091E00081FDFCCF0895C4
:10306000CF92DF92EF92FF920F931F93CF93DF9354
:10307000EC018B017A010E948E19811133C0E11499
:10308000F10439F0F70180819181081B190BC80FF9
:10309000D91FC12CD12C0115110519F18091E8001F
:1030A00085FD16C08091E8008E778093E800E114DA
:1030B000F10449F0F70180819181C80ED91ED182B7
:1030C000C08285E00FC00E948E19882321F30AC0B8
:1030D00089918093F10001501109FFEFCF1ADF0AA7
:1030E000DACF80E0DF91CF911F910F91FF90EF90A9
:1030F000DF90CF9008952091AE023091AF02261755
:10310000370748F06115710539F42091E8002E77F2
:103110002093E80001C0B901FC0120E061157105B0
:1031200079F18091A7028823F1F18530F1F1809146
:10313000E80083FD3CC08091E80082FD2EC08091B4
:10314000E80080FFEBCF2091F3008091F20090E047
:10315000922B6115710551F08830910538F4219159
:103160002093F100615071090196F3CF21E0089797
:1031700009F020E08091E8008E778093E800CECFC0
:103180002111CFCF0AC08091A702882361F085303A
:1031900061F08091E80083FD0AC08091E80082FF21
:1031A000F2CF80E0089582E0089583E0089581E001
:1031B00008952091AE023091AF022617370748F0EC
:1031C0006115710539F42091E8002E772093E8000D
:1031D00001C0B901FC0120E06115710591F18091F8
:1031E000A702882309F440C0853009F43FC08091CC
:1031F000E80083FD3DC08091E80082FD2FC08091F2
:10320000E80080FFE9CF2091F3008091F20090E088
:10321000922B6115710559F08830910540F4249185
:103220002093F1003196615071090196F2CF21E0AF
:10323000089709F020E08091E8008E778093E800FD
:10324000CBCF2111CCCF0AC08091A702882361F097
:10325000853061F08091E80083FD0AC08091E8002C
:1032600082FFF2CF80E0089582E0089583E0089520
:1032700081E00895982F973068F59093E9009817AA
:1032800039F07091EC002091ED005091F00003C0F6
:10329000242F762F50E021FD02C09F5FECCF3091AC
:1032A000EB003E7F3093EB003091ED003D7F30939B
:1032B000ED003091EB0031603093EB007093EC0047
:1032C0002093ED005093F0002091EE0027FDE5CF14
:1032D00080E008958F708093E90081E008958091E7
:1032E000A80287FF11C08091E80082FD05C080918F
:1032F000A7028111F8CF11C08091E8008B770BC035
:103300008091A702882349F08091E80080FFF8CFE0
:103310008091E8008E778093E80008952091E40082
:103320003091E50095E64091EC00842F817040FFDC
:1033300023C08091E80080FD1DC08091A7028823F2
:1033400099F0853099F08091EB0085FD11C0409196
:10335000E4005091E5002417350729F3915011F04E
:103360009A01E1CF84E0089582E0089583E0089512
:1033700081E0089580E008954091E80042FFDDCFAC
:1033800008950E942F1A0E94371AE0EEF0E0808123
:1033900081608083E8EDF0E080818F77808319BCC5
:1033A000A7EDB0E08C918E7F8C9380818F7E80839F
:1033B0001092A60208950F931F93CF93DF930E945C
:1033C0002F1A0E94371AC8EDD0E088818F77888342
:1033D00088818068888388818F7D888319BC10925A
:1033E000A7021092A3021092A5021092A40200EE6E
:1033F00010E0F80180818B7F8083888181608883E1
:1034000042E060E080E00E943A19E1EEF0E0808165
:103410008E7F8083E2EEF0E0808181608083808116
:1034200088608083F80180818E7F808388818061BD
:103430008883DF91CF911F910F910895E8EDF0E01F
:1034400080818F7E8083E7EDF0E0808181608083E2
:1034500084E082BF81E08093A6020C94DB19E8ED42
:10346000F0E080818E7F80831092E20008951092B8
:10347000DA001092E10008951F920F920FB60F929A
:1034800011242F933F934F935F936F937F938F9369
:103490009F93AF93BF93EF93FF938091E10082FFDF
:1034A0000BC08091E20082FF07C08091E1008B7F1A
:1034B0008093E1000E94B21C8091DA0080FF1FC05F
:1034C0008091D80080FF1BC08091DA008E7F8093AE
:1034D000DA008091D90080FF0DC080E189BD82E1D2
:1034E00089BD09B400FEFDCF81E08093A7020E9450
:1034F000841605C019BC1092A7020E9492168091F2
:10350000E10080FF19C08091E20080FF15C080912A
:10351000E2008E7F8093E2008091E20080618093E0
:10352000E2008091D80080628093D80019BC85E0C9
:103530008093A7020E9497168091E10084FF30C01B
:103540008091E20084FF2CC080E189BD82E189BDC9
:1035500009B400FEFDCF8091D8008F7D8093D80004
:103560008091E1008F7E8093E1008091E2008F7E68
:103570008093E2008091E20081608093E20080917C
:10358000A302882311F084E007C08091E30087FD47
:1035900002C081E001C083E08093A7020E949F16D1
:1035A0008091E10083FF29C08091E20083FF25C064
:1035B0008091E100877F8093E10082E08093A70201
:1035C0001092A3028091E1008E7F8093E1008091B0
:1035D000E2008E7F8093E2008091E2008061809320
:1035E000E20042E060E080E00E943A198091F00041
:1035F00088608093F0000E949516FF91EF91BF9133
:10360000AF919F918F917F916F915F914F913F917A
:103610002F910F900FBE0F901F9018951F920F9231
:103620000FB60F9211242F933F934F935F936F9395
:103630007F938F939F93AF93BF93CF93DF93EF933A
:10364000FF93C091E900CF708091EC00D82FD1702A
:1036500080FDD0E81092E9008091F000877F809390
:10366000F00078940E94521B1092E9008091F000C3
:1036700088608093F000CD2BCF70C093E900FF915C
:10368000EF91DF91CF91BF91AF919F918F917F91FA
:103690006F915F914F913F912F910F900FBE0F90BF
:1036A0001F9018951F93CF93DF93CDB7DEB7AA97DE
:1036B0000FB6F894DEBF0FBECDBFE8EAF2E080910E
:1036C000F100819322E0E03BF207C9F70E94BD16AA
:1036D0008091E80083FF2EC18091A8029091A902F9
:1036E000492F50E04A30510508F024C1FA01EE5943
:1036F000FF4F0C94CE1C803821F0823809F01AC19B
:1037000008C08091A4029091A502992389F082605B
:103710000FC08091AC028F70873008F00BC180938E
:10372000E9008091EB0085FB882780F91092E90081
:103730009091E800977F9093E8008093F1001092B9
:10374000F100D1C0282F2D7F09F0F4C0882319F093
:10375000823061F0EFC08091AA02813009F0EAC0A6
:10376000933009F080E08093A5022EC08091AA02D8
:1037700081112AC08091AC028F702FEF280F263064
:1037800008F0D8C08093E9002091EB0020FF1CC016
:10379000933021F48091EB00806214C09091EB0093
:1037A00090619093EB0021E030E0A90102C0440F4A
:1037B000551F8A95E2F74093EA001092EA00809143
:1037C000EB0088608093EB001092E9008091E800A4
:1037D000877F8093E8000E946F19ACC08111AAC056
:1037E0001091AA021F778091E3008078812B80934B
:1037F000E3008091E800877F8093E8000E946F19C2
:103800008091E80080FFFCCF8091E3008068809386
:10381000E300111102C082E001C083E08093A7029F
:1038200089C08058823008F085C08091AA029091AA
:10383000AB028C3D53E0950779F583E08A838AE2F9
:1038400089834FB7F894DE01139620E03EE051E201
:10385000E32FF0E050935700E49120FF03C0E2957E
:10386000EF703F5FEF708E2F90E0EA3010F0C79658
:1038700001C0C0968D939D932F5F243149F74FBFB0
:103880008091E800877F8093E8006AE270E0CE01D3
:1038900001960E947B1816C06091AC027091AD0237
:1038A000AE014F5F5F4F0E94BF17BC01892B09F427
:1038B00041C09091E800977F9093E80089819A81B8
:1038C0000E94D9188091E8008B778093E80032C07D
:1038D000803881F58091E800877F8093E8008091AF
:1038E000A3028093F1008091E8008E7772CF81115E
:1038F00021C08091AA029091AB0299270297D4F43B
:103900008091E800877F8093E8008091AA028093ED
:10391000A3020E946F198091A302811106C08091B9
:10392000E30087FD02C081E001C084E08093A7022C
:103930000E94A9168091E80083FF0AC08091E800E8
:10394000877F8093E8008091EB0080628093EB009A
:10395000AA960FB6F894DEBF0FBECDBFDF91CF9110
:103960001F9108950895CF938091A7028823A1F015
:10397000C091E900CF709091EC00892F817090FD8B
:1039800080E8C82B1092E9008091E80083FD0E9436
:10399000521BCF70C093E900CF910895EE0FFF1F27
:1039A0000590F491E02D0994FB01DC0104C08D9198
:1039B0000190801921F441505040C8F7881B990BA1
:1039C0000895F999FECF92BD81BDF89A992780B5E7
:1039D0000895A8E1B0E042E050E00C94151D262FB8
:1039E000F999FECF92BD81BDF89A019700B40216F5
:1039F00039F01FBA20BD0FB6F894FA9AF99A0FBEA3
:103A000008950396272F0E94F01C0E94EF1C252F7B
:103A10000E94F01C242F0C94F01C0196272F0E946A
:103A2000F01C0C94EF1CDC01CB01FC01F999FECFDA
:103A300006C0F2BDE1BDF89A319600B40D92415036
:0A3A40005040B8F70895F894FFCF46
:103A4A00C80020020B160F1683167F167B160E1659
:103A5A0001E200E900EA00B500B600B700CD008334
:103A6A0001CC008A01920194012102230224022539
:103A7A0002260227022A02B300B4006F00700081F6
:103A8A008283E200E900EA00B500B600B700CD0083
:103A9A008301CC008A0192019401210223022402AB
:103AAA002502260227022A02B300B4006F00700022
:103ABA00818283909192939594969734353666676E
:083ACA00F7F63337303132000A
:00000001FF
